:020000040000FA
:020000001828BE
:0800080008290A30DB00DB0BC4
:100010000A280F282430DC00DC0B0C2807280800F5
:10002000DD00DD0ADD0B1528172805201228080041
:10003000FF23831690008312073099008316FC304B
:1000400085008113FC3095001030960083128B15CB
:100050000B1005108510051A40288514FF3010205C
:10006000051D37287F30A800013090203B287F30C5
:10007000A800003090208510051E3B280430102079
:100080008B17A0200030A80089202002031D7F28A4
:100090007F30A8008920013C031D6D280C3021020F
:1000A0000319572804302102031959287F28A7145F
:1000B0005A282715051D6628A71C6128A7100514B6
:1000C0007F28271D7F28271105107F280514FF3062
:1000D0001020FF30102005107F280C302102031D56
:1000E0007F28051D79280518772805147F28051015
:1000F0007F280514FF301020FF30102005108120CC
:1001000040282830A400851A8128FE20A40B8328CB
:100110000800280883169B001C141A088312080084
:1001200083169A008312280883169B001C155530ED
:100130009D00AA309D009C149C189C2883120800E6
:10014000CD20DE202008A5002108A600CD20DE203D
:1001500020082502031DCC2821082602031DCC28D7
:100160002008A5002108A600CD20DE2020082502B9
:10017000031DCC2821082602031DCC282008A50039
:100180002108A600CD20DE2020082502031DCC2852
:1001900021082602031DCC280800B430A400851ACB
:1001A000CD280321A40BCF280530A400851ED42818
:1001B0000321A40BD628851ADB280800A001A10181
:1001C0000830A300FE200314851A0310A00CA30B13
:1001D000EA28ED28D420FE20E3280430A300D42010
:1001E000FE200314851A0310A10CA30BEF28D420C2
:1001F0000310A10CA10CA10CA10C0800AE30A200B0
:10020000A20B002908001330A200A20B0529080048
:10021000DF000308DE00051A172985140030A80046
:10022000A02020089020051E1329043010200B1058
:0A02300085105E0883005F080900D6
:084000000100090004000900A1
:02400E00A431DB
:024200000700B5
:0242FE000000BE
:00000001FF
